:020000040000FA
:060000002BEF09F01200D5
:020006001200E6
:060008006AEF03F0120094
:02000E000100EF
:0C00100092120000000100009D000000A2
:04001C00D9CFE6FF53
:10002000E1CFD9FF020EE1260101100EA76F0C0EE1
:10003000A86F000EA96F720ED36EC26A0D0EC16E4C
:10004000C06AC30E926E010E936EC50E946E8968DF
:100050008A68FD0E8B6E0D0EE66E040EE66ED90EEE
:10006000E66EC8EC07F0E552E552E552870EE66E03
:10007000EEEC08F0E55247EC09F042EC09F000091B
:1000800001E0FBD739EC09F0F3CF14F0F4CF15F011
:10009000560E0D6E010E0E6E14C008F015C009F05C
:1000A00022EC06F008C014F009C015F014C070F17D
:1000B0008F0EE66EEEEC08F0E55247EC09F042ECEC
:1000C00009F0000901E0FBD739EC09F0F3CF14F097
:1000D000F4CF15F0560E0D6E010E0E6E14C008F022
:1000E00015C009F022EC06F008C014F009C015F0A4
:1000F000030E1502F3CF15F01402F3CF14F0F450F1
:10010000152614500101702770C1E9FFEA6AE9BEA3
:10011000EA68040ED890E936EA36E806FBE1000EFC
:10012000E926010EEA220C0EE926000EEA22EECFA5
:1001300014F0EFCF15F0080E141801E1155022E06D
:10014000040E141801E1155017E0020E141801E115
:1001500015500CE0010E141801E1155001E018D003
:10016000450EE66E46EC08F0E55212D0550EE66EEE
:1001700046EC08F0E5520CD0650EE66E46EC08F051
:10018000E55206D0750EE66E46EC08F0E55200D05A
:10019000000EE66EE66A67EC08F0E552E552B196AD
:1001A000850EE66ED6EC08F0E552BC0EE66EBBECB2
:1001B00008F0E552CC6A70C1E9FFEA6AE9BEEA6874
:1001C000040ED890E936EA36E806FBE1000EE9268F
:1001D000010EEA220E0EE926000EEA22EECF14F0FE
:1001E000EFCF15F0100E141801E1155017E0080EAE
:1001F000141801E115500CE0040E141801E115501B
:1002000001E012D0D10EE66E9FEC08F0E5520CD062
:10021000D20EE66E9FEC08F0E55206D0D30EE66EE5
:100220009FEC08F0E55200D0000EE66EE66A83EC23
:1002300008F0E552E552F288F18CD09E9F849D84AF
:100240009D82F28CF28E8250400B02E0000E01D0B3
:10025000030E0101736F945149E1440ED8809B5500
:10026000000E9C5526E3E66A9BC1E6FF9CC1E6FFB3
:100270007FEC07F0E552E552E5520101AA6F010E4D
:10028000E66E9BC1E6FF9CC1E6FF7FEC07F0E552FE
:10029000E552E5520101AB6F020EE66E9BC1E6FF2F
:1002A0009CC1E6FF7FEC07F0E552E552E552010103
:1002B000AC6F0101500E9B5D000E9C5916E3010EC0
:1002C000946F80AE08D00101B80EA76F090EA86F19
:1002D000000EA96F07D00101E80EA76F0A0EA86FE4
:1002E000000EA96F0101020E7C6FE9D18DC18FF163
:1002F0008EC190F18F51901141E08FC118F090C1E3
:1003000019F01A6A1B6A70C1E9FFEA6AE9BEEA6875
:10031000040ED890E936EA36E806FBE1000EE9263D
:10032000010EEA22060EE926000EEA22EECF14F0B4
:10033000EFCF15F0166A176A060ED89014361536E8
:1003400016361736E806F9E114C006F015C007F0B6
:1003500016C008F017C009F018C00BF019C00CF057
:100360001AC00DF01BC00EF048EC06F006C087F175
:1003700007C088F108C089F109C08AF185C118F069
:1003800086C119F01A6A1B6A70C1E9FFEA6AE9BE00
:10039000EA68040ED890E936EA36E806FBE1000E7A
:1003A000E926010EEA22EECF14F0EECF15F0EECFE3
:1003B00016F0EFCF17F0060ED89014361536163615
:1003C0001736E806F9E114C006F015C007F016C0AC
:1003D00008F017C009F018C00BF019C00CF01AC0D3
:1003E0000DF01BC00EF048EC06F006C081F107C00E
:1003F00082F108C083F109C084F1010193052FE166
:1004000070C1E9FFEA6AE9BEEA68040ED890E936ED
:10041000EA36E806FBE1000EE926010EEA22040EA8
:10042000E926000EEA22EECF14F0EFCF15F0166A9F
:10043000176A15AE02D01668176801018A5117189D
:10044000E8AE02D0173408D01450875D1550885993
:100450001650895917508A5902E2936B31D0935143
:100460002FE170C1E9FFEA6AE9BEEA68040ED8909C
:10047000E936EA36E806FBE1000EE926010EEA223B
:10048000080EE926000EEA22EECF14F0EFCF15F0A9
:10049000166A176A15AE02D0166817681750010160
:1004A0008A19E8AE02D08A3508D08751145C885189
:1004B0001558895116588A51175802E2010E936F48
:1004C000935125E1760EE96E010EEA6EEE50875DDE
:1004D000066EEE508859076EEE508959086EEE5040
:1004E0008A59096E400E0B6E0C6A0D6A0E6A48EC52
:1004F00006F0010176510624766F77510720776F59
:1005000078510820786F79510920796F2BD09305A5
:1005100025E1760EE96E010EEA6EEE50815D066E03
:10052000EE508259076EEE508359086EEE50845992
:10053000096E400E0B6E0C6A0D6A0E6A48EC06F0EE
:10054000010176510624766F77510720776F785135
:100550000820786F79510920796F04D0766B776B1A
:10056000786B796B76C106F077C107F078C108F037
:1005700079C109F0400E0B6E0C6A0D6A0E6A48ECE8
:1005800006F006C074F107C075F1020E0101935D1B
:1005900007E0010E7425746F000E7521756F02D08F
:1005A000746B756B92517519E8AE02D0753504D035
:1005B0007451915D7551925904E274C191F175C104
:1005C00092F1753504E27451DC08050E755502E2AE
:1005D000020E7C6F82BE04D091C174F192C175F19C
:1005E00074C114F075C115F00A0E0D6E0E6A14C0B8
:1005F00008F015C009F022EC06F004C014F005C0A4
:1006000015F014C0AAF10A0E010175AF02D0D890FE
:1006100003D0745D000E755921E374C114F075C1E7
:1006200015F0640E0D6E0E6A14C008F015C009F0C6
:1006300022EC06F004C014F005C015F00A0E0D6E91
:100640000E6A14C008F015C009F022EC06F008C0CC
:1006500014F009C015F014C0ABF103D001010A0E6B
:10066000AB6F640E010175AF02D0D89003D0745DFA
:10067000000E755921E374C114F075C115F0640EB4
:100680000D6E0E6A14C008F015C009F022EC06F0D9
:1006900008C014F009C015F00A0E0D6E0E6A14C0E1
:1006A00008F015C009F022EC06F004C014F005C0F3
:1006B00015F014C0ACF103D001010A0EAC6FC3D524
:1006C000020EE15C02E2E16AE552E16EE552E7CF3B
:1006D000D9FF1200DACFE4FFE2CFDAFFE9CFE4FF7F
:1006E000EACFE4FFF6CFE4FFF7CFE4FFF8CFE4FF73
:1006F000F5CFE4FFF3CFE4FFF4CFE4FFFACFE4FF5C
:10070000FBCFE4FF00EE00F0140EE80403E3EECFAD
:10071000E4FFFBD700EE14F00C0EE80403E3EECF89
:10072000E4FFFBD7E6529EA41CD09E947DC17FF1CE
:100730007EC180F123EC08F0F3CF7DF1F4CF7EF1A0
:1007400001017F517D5D856F80517E59866F9507D0
:10075000000E965B9551961104E18B76010E956F14
:10076000966BF2A22AD0F2928BC18DF18CC18EF1E0
:1007700001018B6B8C6B020E935D1FE197519811F9
:1007800003E0976B986B19D070C1E9FFEA6AE9BE84
:10079000EA68040ED890E936EA36E806FBE1000E76
:1007A000E926010EEA220A0EE926000EEA22EECF21
:1007B0008DF1EDCF8EF10101936BF2A42DD0F29467
:1007C00001018B2B000E8C2370C1E9FFEA6AE9BEA0
:1007D000EA68040ED890E936EA36E806FBE1000E36
:1007E000E926010EEA220A0EE926000EEA22EECFE1
:1007F00020F0EFCF21F0010120508B5D21508C596A
:100800000BE38B6B8C6B876B886B896B8A6B020E2F
:10081000936F010E976F986B9EB09E909EA2A4D08E
:100820009E920101992B000E9A23320ED880995581
:10083000000E9A5505E29B2B000E9C23996B9A6B38
:10084000000EE76E7C19E8AE02D07C3503D0E7508D
:10085000D8807C5518E27A2B000E7B237B3504E28E
:100860007A517808000E7B5504E27A6B7B6B7C072B
:100870000AD07B3504E27A513C08000E7B5502E237
:100880008B9201D08B82712B710512E180AE02D068
:100890008A9201D08B9AAAC1E6FF07D0A9C1FBFFBB
:1008A000A8C1FAFF0101A751F96EF8DFE5525CD04B
:1008B000050ED8807255715D0AE180AE02D08A8241
:1008C00001D08B8A0A0EE66E77D8E5524DD0060E1F
:1008D000715D0EE18B98ABC1E6FF07D0A9C1FBFFAC
:1008E000A8C1FAFF0101A751F96EF8DFE5523CD02B
:1008F0000A0ED8807255715D06E18B880A0EE66E8D
:100900005BD8E55231D00B0E715D12E180AE02D0A2
:100910008B9A01D08A92ACC1E6FF07D0A9C1FBFF38
:10092000A8C1FAFF0101A751F96EF8DFE5521CD00A
:100930000F0ED8807255715D0AE180AE02D08B8AAD
:1009400001D08A820A0EE66E37D8E5520DD00F0E1E
:10095000E76E7119E8AE02D0E73402D0E750715D5E
:1009600003E3716B73C172F1E55200EE1FF00C0EE0
:10097000E80403E3E5CFEDFFFBD700EE13F0140E20
:10098000E80403E3E5CFEDFFFBD7E5CFFBFFE5CFC1
:10099000FAFFE5CFF4FFE5CFF3FFE5CFF5FFE5CFB5
:1009A000F8FFE5CFF7FFE5CFF6FFE5CFEAFFE5CFAC
:1009B000E9FFE5CFDAFF1100D9CFE6FFE1CFD9FF9C
:1009C0003C0E89128A1280AC46D0FE0EDB50090A1A
:1009D0003CE0010A35E00F0A2FE0010A28E0030A93
:1009E00021E0010A1AE0070A13E0010A0CE0030AF9
:1009F00007E0010A01E02ED0C70E89168A162AD018
:100A0000CF0E891627D0E70E8916CB0E8A1622D074
:100A1000C70E8916DB0E8A161DD0CF0E8916F30E6F
:100A20008A1618D0D70E8916D30E8A1613D0D70E71
:100A30008916C30E8A160ED0C70E89168A960AD05A
:100A4000C70E8916C30E8A1605D0C70E8916D30E97
:100A50008A1600D045D0FE0EDB50090A3CE0010AA0
:100A600035E00F0A2FE0010A28E0030A21E0010A1D
:100A70001AE0070A13E0010A0CE0030A07E0010A82
:100A800001E02ED0C70E89168A162AD0CF0E8916FD
:100A900027D0D70E8916D30E8A1622D0C70E8916F4
:100AA000DB0E8A161DD0CF0E8916EB0E8A1618D0D3
:100AB000E70E8916CB0E8A1613D0E70E8916C30EE1
:100AC0008A160ED0CF0E89168A160AD0C70E89163E
:100AD000C30E8A1605D0C70E8916CB0E8A1600D013
:100AE000E552E7CFD9FF1200D9CFE6FFE1CFD9FF1A
:100AF0003C0E89128A1280AC44D0FE0EDB50090AEB
:100B00003AE0010A33E00F0A2DE0010A26E0030A69
:100B10001FE0010A19E0070A13E0010A0CE0030ACA
:100B200007E0010A01E02CD0C70E89168A1628D0EA
:100B3000E70E8A1625D0E70E8916CB0E8A1620D02E
:100B40008996C30E8A161CD0899AE30E8A1618D08D
:100B5000D70E8916D30E8A1613D0C70E8916D30E58
:100B60008A160ED0899AC70E8A160AD0C70E891621
:100B7000C30E8A1605D0D70E8916C30E8A1600D06A
:100B800043D0FE0EDB50090A3AE0010A33E00F0AB7
:100B90002DE0010A26E0030A1FE0010A19E0070A16
:100BA00013E0010A0CE0030A07E0010A01E02CD07F
:100BB000C70E89168A1628D0E70E8A1625D0D70EBA
:100BC0008916D30E8A1620D08996C30E8A161CD099
:100BD0008998E30E8A1618D0E70E8916CB0E8A166E
:100BE00013D0C70E8916CB0E8A160ED0E70E8916C3
:100BF0008A160AD0C70E8916C30E8A1605D0E70ECC
:100C00008916C30E8A1600D0E552E7CFD9FF12002D
:100C1000D9CFE6FFE1CFD9FF3C0E8912FE0EDB50A3
:100C20000F0B040DF31C89163C0E8A12FE0EDB50CE
:100C3000F00BE840E8403F0BE81C8A16E552E7CF8E
:040C4000D9FF1200C6
:0C0C4400006A0EAE2BEF06F00D6C0E1EC9
:100C5000E86A0E22001E09AE33EF06F0086C091E8A
:100C6000E86A0922001E05EC09F009BE43EF06F010
:100C700000AE000C086C091EE86A0922046C051E0F
:100C8000E86A0522000C00BE3AEF06F00188FF0C6E
:100C9000006AE86A0EAE55EF06F00B6C0C1E0D1ED6
:100CA0000E1E0C220D220E22001E09AE60EF06F071
:100CB000066C071E081E091E072208220922001EB4
:100CC000FFEC07F009BE77EF06F000AE000C066CF3
:100CD000071E081E091EE86A072208220922026C64
:100CE000031E041E051E032204220522000C00BE62
:100CF00067EF06F00188FF0C09C013F008C012F07E
:100D000007C011F007500C02F4CF05F0F3CF04F048
:100D100008500D02F4CF07F0F3CF06F00C02F350A9
:100D20000526F4500622E86A072211500D02F350FE
:100D30000526F4500622E86A072209500C02F350F7
:100D40000626F450072209500D02086AE86A0822B4
:100D5000F3500726F450082211500E02F3500626D5
:100D6000F4500722096AE86A0822092212500E028A
:100D7000F3500726F4500822E86A092213500E02A5
:0A0D8000F3500826F4500922000C7D
:060D8A0000000000000063
:100D900000000000000000000002000080020004CB
:100DA0008002300082081482402092080896444055
:100DB000B22108BA0845F25020FB0418FFA050FFEA
:100DC00004D4FF22F0FF01F6FF08F7FF04FFFFA0A5
:100DD000FFFFA8FFFFE4FFFFF4FFFFF6FFFFFEFFAA
:100DE000FFFFFFFFFFFFFFFFFFFFFFFFFFFFFFFF13
:100DF000FFFFFFFFFFFFFFFFFFFFFFFFFFFFFFD929
:100E0000FFFFD9FFFF81D9FF81D9FF8181D981817E
:100E1000D98181818181818181818181818181816A
:100E200081818181818101818100818100808100B6
:100E30000081000001000000000000000000D60C4E
:100E4000EED60CEED60CEED60CEED60CEED60CEEA4
:0F0E5000D60CEED60CEE000000000000000000F3
:100E60000E0EF66E000EF76E000EF86E0101090010
:100E7000F550A26F0900F550A36F03E1A26701D0FE
:100E80003DD00900F5509D6F0900F5509E6F090097
:100E9000F5509F6F09000900F550E96E0900F55003
:100EA000EA6E090009000900F550A06F0900F5502D
:100EB000A16F09000900F6CFA4F1F7CFA5F1F8CF93
:100EC000A6F19DC1F6FF9EC1F7FF9FC1F8FF01018A
:100ED000A05302E1A15307E00900F550EE6EA00710
:100EE000F8E2A107F9D7A4C1F6FFA5C1F7FFA6C193
:0E0EF000F8FF0101A207000EA35BBFD712009E
:020EFE00D9CF4A
:100F0000E6FFE1CFD9FF8A0E176E0D0E186E000EA8
:100F1000196EFD0EDBCF1AF0FE0EDBCF1BF01C6A44
:100F2000030E0C6E0D6A0E6A1AC007F01BC008F0A3
:100F30001CC009F07CEC06F004C01AF005C01BF0E0
:100F400006C01CF017501A24146E18501B20156E82
:100F500019501C20166EFC0EDBCF1DF01E6A1F6A96
:100F60001DAE02D01E681F6814501D24F36E15506C
:100F70001E20F46E16501F20F86EF4CFF7FFF3CF4B
:100F8000F6FF0800F55000D0E552E7CFD9FF120078
:100F9000D9CFE6FFDACFE6FFE1CFD9FFE2CFDAFF24
:100FA000C26AC06AFC0EDB407F0B3C0BC26EFC0EBB
:100FB000DB38F00B300B146EFB0EDB500F0B1410F4
:100FC000C16EFD0EDB50040DF350380B156EFD0E97
:100FD000DB380F0B070B146EFD0EDB50800B14106B
:100FE0001510C06EFC0EDBAE03D09E9C9D8CF28C67
:0E0FF000C280E552E5CFDAFFE7CFD9FF12004D
:020FFE00056A82
:10100000046A036A026A200EE76ED8900636073635
:101010000836093602360336043605360B50025CB4
:101020000C5003580D5004580E50055809E30B504E
:10103000025E0C50035A0D50045A0E50055A062AEF
:06104000E72EE4D71200C8
:0A104600D9CFE6FFDACFE6FFE1CFD5
:10105000D9FFE2CFDAFFE652E6520101AD919EB42C
:10106000AD81BE50DF6E010EBFCFDBFFDECF14F0CF
:10107000DDCF15F014C0F3FF15C0F4FFE552E552C3
:0C108000E552E5CFDAFFE7CFD9FF120000
:04108C00D9CFE6FFD3
:10109000DACFE6FFE1CFD9FFE2CFDAFFFD0EDB507A
:1010A0007E0BCD6EFD0EDBAC02D0CD8E01D0CD9E81
:1010B000CF6ACE6A9E90DBAE02D09D8001D09D901B
:0E10C000CD80E552E5CFDAFFE7CFD9FF120071
:0210CE00D9CF78
:1010D000E6FFDACFE6FFE1CFD9FFE2CFDAFFE65253
:1010E000E652FC0EDBCFDEFFDBCFDDFF010EDB5077
:1010F000CF6EDF50CE6EE552E552E552E5CFDAFF16
:06110000E7CFD9FF120049
:0A110600D9CFE6FFDACFE6FFE1CF14
:10111000D9FFE2CFDAFFE652E652FC0EDBCFDEFF6C
:10112000DBCFDDFF010EDB50D76EDF50D66EE55210
:0E113000E552E552E5CFDAFFE7CFD9FF120016
:02113E00D9CF07
:10114000E6FFDACFE6FFE1CFD9FFE2CFDAFFFD0E0F
:10115000DB507F0BD56ED76AD66AF294FD0EDBAEFC
:1011600002D0F28A01D0F29AD58EE552E5CFDAFFAD
:06117000E7CFD9FF1200D9
:0A117600D9CFE6FFDACFE6FFE1CFA4
:10118000D9FFE2CFDAFFFD0EDB50FB0BCA6ECC6A53
:101190009E92FD0EDBAE02D09D8201D09D92CA844C
:0C11A000E552E5CFDAFFE7CFD9FF1200DF
:0411AC00D9CFE6FFB2
:1011B000DACFE6FFE1CFD9FFE2CFDAFFFD0EDB5059
:1011C0000F0BBD6EFD0EDBAE02D09E949D84948409
:0C11D000E552E5CFDAFFE7CFD9FF1200AF
:0411DC00D9CFE6FF82
:1011E000DACFE6FFE1CFD9FFE2CFDAFFC30EC214B8
:1011F000146EFD0EDB407F0B3C0B1410C26EE552EB
:0A120000E5CFDAFFE7CFD9FF1200B7
:06120A00056A046A100EE3
:10121000E76ED89008360936043605360D50045C62
:101220000E50055805E30D50045E0E50055A082A6D
:06123000E72EF0D71200CA
:0A123600000EF36E00EE00F0030E50
:1012400001D81200EA6002D0EE6AFCD7F350E960E0
:061250001200EE6AFCD75B
:0A12560012EE00F022EE00F0F86A3C
:10126000019C30EC07F003EC00F00EEC00F0FBD733
:0212700012006A
:0E127200C450176E166AC3501610F36E17C0E4
:04128000F4FF120065
:0A128400C250020B01E0010E12003F
:02128E00C2821A
:0212900012004A
:0E12920040420F00E003A1072B05A107020058
:1012A0000400C0C62D00A00BE316C00CE31604001A
:1012B0000800C0C62D00A00BE316C00CE316020008
:1012C000040080841E00C007420F550A420F02002E
:1012D000040060E31600E005720BD507720B0200F4
:1012E0000400804F1200C004280955062809020096
:1012F000040040420F00E003A1072B05A1070200F4
:1013000004000000000000000000000000000500D4
:1013100000000000000000FFFF00000000000000CF
:0F132000000000000002000100010000000000BA
:020000040030CA
:0100010008F6
:0100020019E4
:010003001EDE
:0100050000FA
:010006008079
:010008000FE8
:01000900C036
:01000A000FE6
:01000B00E014
:01000C000FE4
:01000D0040B2
:00000001FF
